:1000000000308A00E32800000A108A100A118207D3
:1000100028340C34013406340A108A100A1182077D
:10002000413468346F346A340A3444346934733484
:1000300070346C34613479342034663475346E3401
:10004000673475346A3465342034003423308400D6
:100050008313000803193A280130F800F701F70B61
:100060002F28F80B2E284A30F700F70B35283828B0
:10007000800B2C28003407080F39AA00290EF7003E
:10008000F030F7057708F0392A0487000614831644
:100090000610000083120610831606108312003427
:1000A000A708031D55288610562886148316861027
:1000B0008312A80E2808A9003B20A80E2808A90032
:1000C0003B200D30F700F70B632800341430A300F9
:1000D00026200F308316870583128610831686101C
:1000E00083120610831606108312A1012108023C18
:1000F000031C82280230A30026200330A9003B20E5
:10010000A10A76280D30F700F70B84280230A900E9
:100110003B200D30F700F70B8B28A1012108023C92
:10012000031C9E2821080420A200A7012208A80081
:1001300050200230A3002620A10A8E281B2901305E
:100140002302A5002408023C031DA8284030A5076F
:1001500025088038A600A7012608A80050200034F2
:1001600022080C3A0319BE28063A0319C628073A92
:100170000319CC28053A0319D128D628A701013044
:10018000A80050200230A3002620E2280130A3005E
:100190000230A4009F20E2280130A300A4009F2089
:1001A000E228A7011030A8005020E22822081F3CB6
:1001B000031CDC280730A2050130A7002208A80094
:1001C0005020E2282529840183131F3083058316DC
:1001D0001F149F141F159F11FF308312A000831658
:1001E0001F149F141F159F1183121F1083160912CD
:1001F00083129412A01220088316870083122016FF
:100200002008831687008312A01120088316870018
:10021000003083129400831694000108C73908380F
:100220008100831290010030F800920000308316A4
:100230009200831266286430A3002620A1012108C1
:100240000C20A10AF700A200B02815302102031DDE
:060250001F291B296300B9
:02400E00393F38
:00000001FF
